:1000000012C02CC02BC02AC029C028C027C026C0BF
:1000100042C025C023C022C021C020C01FC01EC0B6
:100020001DC01CC01BC011241FBECFE5D4E0DEBF25
:10003000CDBF11E0A0E6B0E0E6EBFEE002C0059027
:100040000D92AC38B107D9F711E0ACE8B1E001C0CE
:100050001D92A639B107E1F75FD02BC7D1CF1F9210
:100060000F920FB60F9211248F938CEE82BFC19B1B
:1000700006C012BAC198C09A8091940105C012BA04
:10008000C098C19A8091930182BB8F910F900FBE4F
:100090000F901F9018951F920F920FB60F92112478
:1000A0008F93809160008DBD809161008CBD8091A7
:1000B0009201882321F480918C0185BB05C0809139
:1000C0009201813009F415BA809192018F5F80937B
:1000D0009201809192018A3011F4109292018F91D5
:1000E0000F900FBE0F901F901895882361F4B3995D
:1000F00002C081E00895B49902C082E00895B599E4
:1001000002C083E0089580E00895B39BFECFB49BC6
:10011000FCCFB59BFACF0895EF92FF920F931F93F8
:10012000CF93DF9389E08093950180938D018FEFCA
:1001300084BB81BB93E097BB8CEF88BB12BAC0989D
:10014000C19A1092920190938C0180E090E4A3E612
:10015000B4E480938E0190938F01A0939001B093AB
:10016000910160918E0170918F0180919001909129
:10017000910120E030E040E051ECC4D220E030E0DA
:1001800040E857E498D20DD4DC01CB01292F332766
:1001900027FD3A952093600060E071E0EFD58093F1
:1001A000610095E099BF8CEE82BF93BF789480ED9B
:1001B00097E028EC30E0F9013197F1F70197D9F792
:1001C0001092930186EB8093940185E085BB80EDCE
:1001D00097E028EC30E0F9013197F1F70197D9F772
:1001E00086EB809393018CE78093940182E085BB3A
:1001F00080ED97E028EC30E0F9013197F1F70197B5
:10020000D9F78CE78093930188E38093940187E08A
:1002100085BB80ED97E028EC30E0F9013197F1F7EC
:100220000197D9F788E3809393018093940115BADD
:1002300080ED97E028EC30E0F9013197F1F7019774
:10024000D9F788E3809393018AEF8093940185E046
:1002500085BB80ED97E028EC30E0F9013197F1F7AC
:100260000197D9F78AEF809393011092940182E06D
:1002700085BB80ED97E028EC30E0F9013197F1F78C
:100280000197D9F7109293011092940187E085BBF2
:1002900080ED97E028EC30E0F9013197F1F7019714
:1002A000D9F715BA84E0809393018093940181E09B
:1002B0008EBD809160008DBD809161008CBD82E01B
:1002C00090E0C0E0D0E053E0E52E47E0F42E08ECEB
:1002D00010E0009709F464C08330910509F451C01F
:1002E000019729F4C530D1052CF4219603C020973D
:1002F00009F02197FE01EE59FF4F81818093930110
:10030000FE01EE0FFF1FEE0FFF1FE459FF4F82812A
:100310008093940120813181442737FD4095542FEB
:1003200060E472E48FE090E03CD5CA01B901DFD20D
:1003300060938E0170938F0180939001909391014F
:1003400060918E0170918F01809190019091910147
:1003500020E030E040E051ECD5D120E030E040E852
:1003600057E4A9D11ED3DC01CB01292F332727FD68
:100370003A952093600060E071E000D580936100C1
:1003800009C080918C01833019F4F0928C0102C075
:10039000E0928C01B39BFECFB49BFCCFB59BFACF10
:1003A00084EF91E0F8013197F1F70197D9F7B3990C
:1003B00002C081E009C0B49902C082E005C0B59BCB
:1003C00002C080E001C083E090E083CFA0E0B0E015
:1003D000EBEEF1E037C5DC012B01FA019C91923084
:1003E00008F439C1EB018881823008F433C19430BC
:1003F00069F4843009F02FC111969C91119789817D
:10040000981709F428C1A4E8B0E025C1843009F4A4
:1004100021C18230A9F4923009F01DC19A01AD01C9
:1004200088E0EA010990AE01E90109929E0181503C
:10043000C1F7E201898111969C918923818308C1CA
:10044000923009F407C112962D903C901397EB015E
:100450008A819B811496AD90BD90CD90DC901797CA
:10046000EC80FD800E811F819101281B390BB901A1
:1004700037FF04C066277727621B730B6032710554
:100480000CF061C0121613066CF537014801062EF8
:1004900004C096948794779467940A94D2F721E0E5
:1004A00030E040E050E004C0220F331F441F551FCE
:1004B0006A95D2F721503040404050402E213F21D4
:1004C00040235123211531054105510521F021E03B
:1004D00030E040E050E079018A01E628F728082959
:1004E00019293CC0232BD1F1260E371E35014601B8
:1004F000062E04C096948794779467940A94D2F752
:1005000021E030E040E050E004C0220F331F441FE0
:10051000551F6A95D2F721503040404050402A2163
:100520003B214C215D21211531054105510521F06B
:1005300021E030E040E050E059016A01A628B728E8
:10054000C828D9280BC0821593052CF01C01AA24B9
:10055000BB24650103C0EE24FF24870111969C9102
:10056000D20111968C91981709F445C0992339F05E
:10057000A80197012A193B094C095D0906C0A6018B
:1005800095012E193F09400B510B57FD08C01182F0
:100590003382228224833583468357831DC081E0C2
:1005A00081833382228288279927DC01821B930B67
:1005B000A40BB50B84839583A683B7830DC0220F4C
:1005C000331F441F551F24833583468357838281FD
:1005D000938101979383828324813581468157815A
:1005E000DA01C9010197A109B1098F5F9F4FAF4F90
:1005F000BF4328F30BC0918333822282EA0CFB1C99
:100600000C1D1D1DE482F5820683178383E0808321
:10061000248135814681578157FF1AC0C901AA2715
:1006200097FDA095BA2F81709070A070B07056950C
:10063000479537952795822B932BA42BB52B848335
:100640009583A683B7838281938101969383828366
:10065000DF0101C0D201CD01CDB7DEB7E2E10EC4AA
:10066000A0E2B0E0E5E3F3E0F9C369837A838B832A
:100670009C832D833E834F835887E9E0EE2EF12C37
:10068000EC0EFD1ECE010196B70100D38E010F5E68
:100690001F4FCE010596B801F9D28A8991E08927CA
:1006A0008A8BC701B801AE01475E5F4F8FDE19D25A
:1006B000A096E6E0EFC3A0E2B0E0E0E6F3E0CEC350
:1006C00069837A838B839C832D833E834F835887F2
:1006D000F9E0EF2EF12CEC0EFD1ECE010196B701D4
:1006E000D5D28E010F5E1F4FCE010596B801CED236
:1006F000C701B801AE01475E5F4F68DEF2D1A09638
:10070000E6E0C8C3A0E2B0E0E7E8F3E09BC369839A
:100710007A838B839C832D833E834F835887CE01BE
:100720000196BE01675F7F4FB1D2CE010596BE0133
:100730006F5E7F4FABD29985923088F08989823085
:10074000C8F0943019F4823051F404C0843029F494
:10075000923081F484E890E0C6C0923049F420E001
:100760009A858A89981321E02A87CE010996BBC011
:10077000823049F420E09A858A89981321E02A8BF7
:10078000CE014196B0C02D843E844F8458886D8838
:100790007E888F88988CEE24FF248701AA24BB24AE
:1007A000650140E050E060E070E0E0E0F0E0C101B1
:1007B00081709070892BE9F0E60CF71C081D191D5B
:1007C0009A01AB012A0D3B1D4C1D5D1D80E090E0A0
:1007D000A0E0B0E0E614F7040805190520F481E074
:1007E00090E0A0E0B0E0BA01A901480F591F6A1FCC
:1007F0007B1FAA0CBB1CCC1CDD1C97FE08C081E033
:1008000090E0A0E0B0E0A82AB92ACA2ADB2A3196F3
:10081000E032F10549F0660C771C881C991C56944F
:10082000479437942794C3CFFA85EA892B893C896A
:100830008B859C85280F391F2E5F3F4F17C0CA013B
:1008400081709070892B61F016950795F794E79465
:1008500080E090E0A0E0B0E8E82AF92A0A2B1B2B00
:1008600076956795579547952F5F3F4F77FDE7CF73
:100870000CC0440F551F661F771F17FD4160EE0C1B
:10088000FF1C001F111F21503040403090E05907DD
:1008900090E0690790E4790760F32B8F3C8FDB01D0
:1008A000CA018F779070A070B07080349105A10557
:1008B000B10561F447FD0AC0E114F1040105110519
:1008C00029F0405C5F4F6F4F7F4F40781A8EFE17C4
:1008D00011F081E08A8F4D8F5E8F6F8F78A383E058
:1008E000898FCE014996FDD0A096E2E1C7C2A8E06B
:1008F000B0E0ECE7F4E0AFC29B01AC0183E0898398
:10090000DA01C9018827B7FD83959927AA27BB2754
:10091000B82E211531054105510519F482E089836E
:1009200039C08823A9F0203080E0380780E04807EC
:1009300080E8580729F460E070E080E09FEC2EC06A
:10094000EE24FF248701E21AF30A040B150B02C000
:1009500079018A018EE1C82ED12CDC82CB82ED8216
:10096000FE820F831887C801B7016CD00197181653
:10097000190684F4082E04C0EE0CFF1C001F111F82
:100980000A94D2F7ED82FE820F831887C81AD90A1B
:10099000DC82CB82BA82CE010196A3D02896E9E010
:1009A00076C2ACE0B0E0E6EDF4E05CC269837A8345
:1009B0008B839C83CE010196BE016B5F7F4F66D116
:1009C0008D81823061F1823050F1843021F48E814A
:1009D000882351F12EC02F81388537FD20C06E81CC
:1009E0002F3131051CF06623F9F023C08EE190E031
:1009F000821B930B29853A854B855C8504C05695EF
:100A00004795379527958A95D2F76623B1F050958B
:100A10004095309521953F4F4F4F5F4F0EC020E0DE
:100A200030E040E050E009C02FEF3FEF4FEF5FE7CD
:100A300004C020E030E040E050E8B901CA012C9643
:100A4000E2E02CC2EF92FF920F931F937B018C0187
:100A500080E0E81680E0F80681E0080780E01807EB
:100A600088F48FEFE816F1040105110531F028F044
:100A700088E090E0A0E0B0E017C080E090E0A0E067
:100A8000B0E012C080E0E81680E0F80680E00807D9
:100A900081E0180728F088E190E0A0E0B0E004C011
:100AA00080E190E0A0E0B0E020E230E040E050E003
:100AB000281B390B4A0B5B0B04C016950795F7945E
:100AC000E7948A95D2F7F701E457FF4F8081281BFE
:100AD000310941095109C9011F910F91FF90EF9010
:100AE0000895DF92EF92FF920F931F93FC01E48031
:100AF000F58006811781D1808081823048F480E0C2
:100B000090E0A0E1B0E0E82AF92A0A2B1B2BA5C04F
:100B1000843009F49FC0823021F4EE24FF24870141
:100B200005C0E114F1040105110519F4E0E0F0E05D
:100B300096C0628173819FEF623879070CF05BC0C9
:100B400022E83FEF261B370B2A3131052CF020E03D
:100B500030E040E050E02AC0B801A701022E04C0F6
:100B600076956795579547950A94D2F781E090E07E
:100B7000A0E0B0E004C0880F991FAA1FBB1F2A95F0
:100B8000D2F70197A109B1098E219F21A023B1239A
:100B90000097A105B10521F081E090E0A0E0B0E070
:100BA0009A01AB01282B392B4A2B5B2BDA01C901A7
:100BB0008F779070A070B07080349105A105B10559
:100BC00039F427FF09C0205C3F4F4F4F5F4F04C0EF
:100BD000215C3F4F4F4F5F4FE0E0F0E02030A0E05E
:100BE0003A07A0E04A07A0E45A0710F0E1E0F0E07D
:100BF00079018A0127C06038710564F5FB01E1586D
:100C0000FF4FD801C7018F779070A070B07080340B
:100C10009105A105B10539F4E7FE0DC080E490E02F
:100C2000A0E0B0E004C08FE390E0A0E0B0E0E80E08
:100C3000F91E0A1F1B1F17FF05C016950795F7948D
:100C4000E794319687E016950795F794E7948A958F
:100C5000D1F705C0EE24FF248701EFEFF0E06E2FFF
:100C6000679566276795902F9F77D794DD24D79453
:100C70008E2F8695492F462B582F5D29B701CA0123
:100C80001F910F91FF90EF90DF900895FC01DB0121
:100C9000408151812281622F6F7770E0221F2227CD
:100CA000221F9381892F880F822B282F30E0991FD4
:100CB0009927991F11969C93119721153105A9F534
:100CC000411551056105710511F482E037C082E8D4
:100CD0009FEF13969C938E9312979A01AB0167E056
:100CE000220F331F441F551F6A95D1F783E08C9361
:100CF0000DC0220F331F441F551F12968D919C91DA
:100D00001397019713969C938E931297203080E04F
:100D1000380780E0480780E4580758F314962D936D
:100D20003D934D935C93179708952F3F310579F4C8
:100D3000411551056105710519F484E08C930895FE
:100D400064FF03C081E08C9312C01C9210C02F5727
:100D5000304013963C932E93129783E08C9387E058
:100D6000440F551F661F771F8A95D1F7706414963C
:100D70004D935D936D937C931797089597FB092E80
:100D800007260AD077FD04D027D006D000201AF419
:100D9000709561957F4F0895F6F7909581959F4FD7
:100DA000089597FB092E05260ED057FD04D028D0B4
:100DB0000AD0001C38F450954095309521953F4F4E
:100DC0004F4F5F4F0895F6F7909580957095619518
:100DD0007F4F8F4F9F4F0895AA1BBB1B51E107C048
:100DE000AA1FBB1FA617B70710F0A61BB70B881FBB
:100DF000991F5A95A9F780959095BC01CD0108954A
:100E0000A1E21A2EAA1BBB1BFD010DC0AA1FBB1F0E
:100E1000EE1FFF1FA217B307E407F50720F0A21B80
:100E2000B30BE40BF50B661F771F881F991F1A94ED
:100E300069F760957095809590959B01AC01BD0117
:100E4000CF0108952F923F924F925F926F927F92BF
:100E50008F929F92AF92BF92CF92DF92EF92FF92CA
:100E60000F931F93CF93DF93CDB7DEB7CA1BDB0B76
:100E70000FB6F894DEBF0FBECDBF09942A8839881B
:100E800048885F846E847D848C849B84AA84B98422
:100E9000C884DF80EE80FD800C811B81AA81B9812E
:100EA000CE0FD11D0FB6F894DEBF0FBECDBFED0142
:060EB0000895F894FFCF45
:100EB6000BDCFA82DCCEA66E7EC2FEEE38037C0028
:100EC6004C04F600BC059E00A8077A00A5093E0062
:100ED600E00C7C000000000000000000000102029F
:100EE60003030303040404040404040405050505BC
:100EF6000505050505050505050505050606060698
:100F0600060606060606060606060606060606067B
:100F16000606060606060606060606060707070767
:100F2600070707070707070707070707070707074B
:100F3600070707070707070707070707070707073B
:100F4600070707070707070707070707070707072B
:100F56000707070707070707070707070808080817
:100F660008080808080808080808080808080808FB
:100F760008080808080808080808080808080808EB
:100F860008080808080808080808080808080808DB
:100F960008080808080808080808080808080808CB
:100FA60008080808080808080808080808080808BB
:100FB60008080808080808080808080808080808AB
:100FC600080808080808080808080808080808089B
:0C0FD600080808080808080808080808AF
:00000001FF
